 dvfc_mc34704

 Timestamp is 4fb05c6b (Mon May 14 13:14:19 2012)

 Preferred load address is 10000000

 Start         Length     Name                   Class
 0001:00000000 00000004H .CRT$XCA                CODE
 0001:00000004 00000004H .CRT$XCZ                CODE
 0001:00000008 00000004H .CRT$XIA                CODE
 0001:0000000c 00000004H .CRT$XIZ                CODE
 0001:00000010 00000004H .CRT$XPA                CODE
 0001:00000014 00000004H .CRT$XPZ                CODE
 0001:00000018 00000004H .CRT$XTA                CODE
 0001:0000001c 00000004H .CRT$XTZ                CODE
 0001:00000020 00000b66H .rdata                  CODE
 0001:00000b88 00000029H .rdata$debug            CODE
 0001:00000bb4 000026bcH .text                   CODE
 0001:00003270 0000005cH .xdata                  CODE
 0001:000032cc 00000050H .idata$2                CODE
 0001:0000331c 00000014H .idata$3                CODE
 0001:00003330 000000b8H .idata$4                CODE
 0001:000033e8 000000ceH .idata$6                CODE
 0001:000034c0 00000098H .edata                  CODE
 0002:00000000 000000b8H .idata$5                DATA
 0002:000000b8 00000064H .data                   DATA
 0002:0000011c 00000060H .bss                    DATA
 0003:00000000 00000198H .pdata                  DATA

  Address         Publics by Value              Rva+Base       Lib:Object

 0000:00000000       ___safe_se_handler_table   00000000     <absolute>
 0000:00000000       ___safe_se_handler_count   00000000     <absolute>
 0001:00000000       __xc_a                     10001000     corelib0:crt0init.obj
 0001:00000004       __xc_z                     10001004     corelib0:crt0init.obj
 0001:00000008       __xi_a                     10001008     corelib0:crt0init.obj
 0001:0000000c       __xi_z                     1000100c     corelib0:crt0init.obj
 0001:00000010       __xp_a                     10001010     corelib0:crt0init.obj
 0001:00000014       __xp_z                     10001014     corelib0:crt0init.obj
 0001:00000018       __xt_a                     10001018     corelib0:crt0init.obj
 0001:0000001c       __xt_z                     1000101c     corelib0:crt0init.obj
 0001:000000d0       ??_C@_1EO@MKMOBHO@?$AAP?$AAm?$AAi?$AAc?$AAR?$AAe?$AAg?$AAu?$AAl?$AAa?$AAt?$AAo?$AAr?$AAG?$AAe?$AAt?$AAV?$AAo?$AAl?$AAt?$AAa?$AAg?$AAe?$AAL?$AAe?$AAv?$AAe?$AAl?$AA?5?$AAf?$AAa?$AAi@ 100010d0     voltctrl.obj
 0001:00000120       ??_C@_1CG@BAGCAEII@?$AAP?$AAm?$AAi?$AAc?$AAO?$AAp?$AAe?$AAn?$AA?5?$AAf?$AAa?$AAi?$AAl?$AAe?$AAd?$AA?$CB?$AA?$AN?$AA?6?$AA?$AA@ 10001120     voltctrl.obj
 0001:00000148       ??_C@_1CI@OHCJFJPM@?$AAE?$AAR?$AAR?$AAO?$AAR?$AA?3?$AA?5?$AA?$CF?$AAs?$AA?5?$AAl?$AAi?$AAn?$AAe?$AA?5?$AA?$CF?$AAd?$AA?3?$AA?5?$AA?$AA@ 10001148     voltctrl.obj
 0001:00000170       ??_C@_1KE@GCFKHLGL@?$AAC?$AA?3?$AA?2?$AAW?$AAI?$AAN?$AAC?$AAE?$AAR?$AAO?$AAO?$AAT?$AAS?$AA?2?$AAT?$AAo?$AAp?$AAa?$AAz?$AA?2?$AAW?$AAI?$AAN?$AAC?$AAE?$AA6?$AA0?$AA0?$AA?2?$AAP?$AAL?$AAA@ 10001170     voltctrl.obj
 0001:00000218       ??_C@_1EI@DKJCDIHI@?$AAC?$AAr?$AAe?$AAa?$AAt?$AAe?$AAT?$AAh?$AAr?$AAe?$AAa?$AAd?$AA?5?$AAf?$AAa?$AAi?$AAl?$AAe?$AAd?$AA?5?$AAf?$AAo?$AAr?$AA?5?$AAD?$AAV?$AAF?$AAC?$AA?5?$AAI?$AAS?$AAT@ 10001218     dvfc_common_topaz_v1:dvfc.obj
 0001:00000260       ??_C@_1CM@KJADCGLN@?$AAB?$AAS?$AAP?$AAD?$AAv?$AAf?$AAc?$AAI?$AAn?$AAi?$AAt?$AA?5?$AAf?$AAa?$AAi?$AAl?$AAe?$AAd?$AA?$CB?$AA?$AN?$AA?6?$AA?$AA@ 10001260     dvfc_common_topaz_v1:dvfc.obj
 0001:00000290       ??_C@_1FO@DKILBGK@?$AAI?$AAn?$AAt?$AAe?$AAr?$AAr?$AAu?$AAp?$AAt?$AAI?$AAn?$AAi?$AAt?$AAi?$AAa?$AAl?$AAi?$AAz?$AAe?$AA?5?$AAf?$AAa?$AAi?$AAl?$AAe?$AAd?$AA?5?$AAf?$AAo?$AAr?$AA?5?$AAD@ 10001290     dvfc_common_topaz_v1:dvfc.obj
 0001:000002f0       ??_C@_1GC@FHBKPEO@?$AAI?$AAO?$AAC?$AAT?$AAL?$AA_?$AAH?$AAA?$AAL?$AA_?$AAR?$AAE?$AAQ?$AAU?$AAE?$AAS?$AAT?$AA_?$AAS?$AAY?$AAS?$AAI?$AAN?$AAT?$AAR?$AA?5?$AAf?$AAa?$AAi?$AAl?$AAe?$AAd@ 100012f0     dvfc_common_topaz_v1:dvfc.obj
 0001:00000358       ??_C@_1FE@KIHGNMCK@?$AAC?$AAr?$AAe?$AAa?$AAt?$AAe?$AAE?$AAv?$AAe?$AAn?$AAt?$AA?5?$AAf?$AAa?$AAi?$AAl?$AAe?$AAd?$AA?5?$AAf?$AAo?$AAr?$AA?5?$AAD?$AAV?$AAF?$AAC?$AA?5?$AAI?$AAS?$AAT?$AA?5@ 10001358     dvfc_common_topaz_v1:dvfc.obj
 0001:000003ac       ??_C@_1CA@DNJNIIBE@?$AAI?$AAN?$AAT?$AAR?$AA_?$AAE?$AAV?$AAE?$AAN?$AAT?$AA_?$AAD?$AAV?$AAF?$AAC?$AA?$AA@ 100013ac     dvfc_common_topaz_v1:dvfc.obj
 0001:000003cc       ??_C@_1DE@BLFOHFK@?$AAR?$AAe?$AAg?$AAQ?$AAu?$AAe?$AAr?$AAy?$AAV?$AAa?$AAl?$AAu?$AAe?$AAE?$AAx?$AA?5?$AAf?$AAa?$AAi?$AAl?$AAe?$AAd?$AA?$CB?$AA?$AN?$AA?6?$AA?$AA@ 100013cc     dvfc_common_topaz_v1:dvfc.obj
 0001:00000400       ??_C@_1M@EENNDIOJ@?$AAI?$AAn?$AAd?$AAe?$AAx?$AA?$AA@ 10001400     dvfc_common_topaz_v1:dvfc.obj
 0001:0000040c       ??_C@_1DA@NAMEIHJM@?$AAO?$AAp?$AAe?$AAn?$AAD?$AAe?$AAv?$AAi?$AAc?$AAe?$AAK?$AAe?$AAy?$AA?5?$AAf?$AAa?$AAi?$AAl?$AAe?$AAd?$AA?$CB?$AA?$AN?$AA?6?$AA?$AA@ 1000140c     dvfc_common_topaz_v1:dvfc.obj
 0001:00000440       ??_C@_1KG@HFLEOAJH@?$AAC?$AA?3?$AA?2?$AAW?$AAI?$AAN?$AAC?$AAE?$AAR?$AAO?$AAO?$AAT?$AAS?$AA?2?$AAT?$AAo?$AAp?$AAa?$AAz?$AA?2?$AAW?$AAI?$AAN?$AAC?$AAE?$AA6?$AA0?$AA0?$AA?2?$AAP?$AAL?$AAA@ 10001440     dvfc_common_topaz_v1:dvfc.obj
 0001:000004e8       ??_C@_1EC@EEIKCCIH@?$AAU?$AAn?$AAs?$AAu?$AAp?$AAp?$AAo?$AAr?$AAt?$AAe?$AAd?$AA?5?$AAD?$AAV?$AAF?$AAC?$AA?5?$AAI?$AAO?$AAC?$AAT?$AAL?$AA?5?$AAc?$AAo?$AAd?$AAe?$AA?5?$AA?$CF?$AAu?$AA?$AN?$AA?6@ 100014e8     dvfc_common_topaz_v1:dvfc.obj
 0001:00000530       ??_C@_1EI@MGFJEBDP@?$AAE?$AAx?$AAc?$AAe?$AAp?$AAt?$AAi?$AAo?$AAn?$AA?5?$AAi?$AAn?$AA?5?$AAD?$AAV?$AAF?$AAC?$AA?5?$AAI?$AAO?$AAC?$AAT?$AAL?$AA_?$AAP?$AAO?$AAW?$AAE?$AAR?$AA_?$AAS?$AAE@ 10001530     dvfc_common_topaz_v1:dvfc.obj
 0001:00000578       ??_C@_1FK@CFOKMKHC@?$AAE?$AAx?$AAc?$AAe?$AAp?$AAt?$AAi?$AAo?$AAn?$AA?5?$AAi?$AAn?$AA?5?$AAD?$AAV?$AAF?$AAC?$AA?5?$AAI?$AAO?$AAC?$AAT?$AAL?$AA_?$AAP?$AAO?$AAW?$AAE?$AAR?$AA_?$AAC?$AAA@ 10001578     dvfc_common_topaz_v1:dvfc.obj
 0001:00000668       ??_C@_1DE@PEIHFJNG@?$AAB?$AAS?$AAP?$AAD?$AAv?$AAf?$AAc?$AAP?$AAo?$AAw?$AAe?$AAr?$AAS?$AAe?$AAt?$AA?5?$AAf?$AAa?$AAi?$AAl?$AAe?$AAd?$AA?$CB?$AA?$AN?$AA?6?$AA?$AA@ 10001668     dvfc:dvfc.obj
 0001:000006a0       ??_C@_1EE@OFPACOHL@?$AAD?$AAv?$AAf?$AAc?$AAI?$AAn?$AAi?$AAt?$AAV?$AAo?$AAl?$AAt?$AAa?$AAg?$AAe?$AAS?$AAu?$AAp?$AAp?$AAl?$AAi?$AAe?$AAs?$AA?5?$AAf?$AAa?$AAi?$AAl?$AAe?$AAd?$AA?$CB?$AA?$AN@ 100016a0     dvfc:dvfc.obj
 0001:000006e8       ??_C@_1FM@FLIAFKCL@?$AAC?$AAr?$AAe?$AAa?$AAt?$AAe?$AAT?$AAh?$AAr?$AAe?$AAa?$AAd?$AA?5?$AAf?$AAa?$AAi?$AAl?$AAe?$AAd?$AA?5?$AAf?$AAo?$AAr?$AA?5?$AAD?$AAV?$AAF?$AAC?$AA?5?$AAw?$AAo?$AAr@ 100016e8     dvfc:dvfc.obj
 0001:00000744       ??_C@_1CE@KCPPCGKP@?$AAE?$AAV?$AAE?$AAN?$AAT?$AA_?$AAD?$AAV?$AAF?$AAC?$AA_?$AAW?$AAO?$AAR?$AAK?$AAE?$AAR?$AA?$AA@ 10001744     dvfc:dvfc.obj
 0001:00000768       ??_C@_1CM@PPPGIKAO@?$AAC?$AAr?$AAe?$AAa?$AAt?$AAe?$AAE?$AAv?$AAe?$AAn?$AAt?$AA?5?$AAf?$AAa?$AAi?$AAl?$AAe?$AAd?$AA?$CB?$AA?$AN?$AA?6?$AA?$AA@ 10001768     dvfc:dvfc.obj
 0001:00000794       ??_C@_1BO@ICEODACO@?$AAE?$AAV?$AAE?$AAN?$AAT?$AA_?$AAS?$AAE?$AAT?$AAP?$AAO?$AAI?$AAN?$AAT?$AA?$AA@ 10001794     dvfc:dvfc.obj
 0001:000007b4       ??_C@_1CO@FMOECGMA@?$AAM?$AAm?$AAM?$AAa?$AAp?$AAI?$AAo?$AAS?$AAp?$AAa?$AAc?$AAe?$AA?5?$AAf?$AAa?$AAi?$AAl?$AAe?$AAd?$AA?$CB?$AA?$AN?$AA?6?$AA?$AA@ 100017b4     dvfc:dvfc.obj
 0001:000007e8       ??_C@_1JK@COCOHCPO@?$AAC?$AA?3?$AA?2?$AAW?$AAI?$AAN?$AAC?$AAE?$AAR?$AAO?$AAO?$AAT?$AAS?$AA?2?$AAT?$AAo?$AAp?$AAa?$AAz?$AA?2?$AAW?$AAI?$AAN?$AAC?$AAE?$AA6?$AA0?$AA0?$AA?2?$AAP?$AAL?$AAA@ 100017e8     dvfc:dvfc.obj
 0001:00000918       ??_C@_1M@LCEEOPDH@?$AAI?$AA2?$AAC?$AA1?$AA?3?$AA?$AA@ 10001918     pmicsdk:mc34704sdk.obj
 0001:00000924       ??_C@_1DC@HNHAGOEA@?$AA?5?$AAR?$AAe?$AAg?$AAu?$AAl?$AAa?$AAt?$AAo?$AAr?$AA?5?$AAn?$AAo?$AAt?$AA?5?$AAs?$AAu?$AAp?$AAp?$AAo?$AAr?$AAt?$AAe?$AAd?$AA?$AA@ 10001924     pmicsdk:mc34704sdk.obj
 0001:00000958       ??_C@_1EO@LPFNDCLA@?$AAR?$AAe?$AAg?$AAu?$AAl?$AAa?$AAt?$AAo?$AAr?$AA?5?$AA8?$AA?5?$AAm?$AAa?$AAn?$AAa?$AAg?$AAe?$AAm?$AAe?$AAn?$AAt?$AA?5?$AAn?$AAo?$AAt?$AA?5?$AAi?$AAm?$AAp?$AAl?$AAe@ 10001958     pmicsdk:mc34704sdk.obj
 0001:000009a8       ??_C@_1EO@KLNCGMFD@?$AAR?$AAe?$AAg?$AAu?$AAl?$AAa?$AAt?$AAo?$AAr?$AA?5?$AA7?$AA?5?$AAm?$AAa?$AAn?$AAa?$AAg?$AAe?$AAm?$AAe?$AAn?$AAt?$AA?5?$AAn?$AAo?$AAt?$AA?5?$AAi?$AAm?$AAp?$AAl?$AAe@ 100019a8     pmicsdk:mc34704sdk.obj
 0001:000009f8       ??_C@_1EO@OBBFGDMA@?$AAR?$AAe?$AAg?$AAu?$AAl?$AAa?$AAt?$AAo?$AAr?$AA?5?$AA6?$AA?5?$AAm?$AAa?$AAn?$AAa?$AAg?$AAe?$AAm?$AAe?$AAn?$AAt?$AA?5?$AAn?$AAo?$AAt?$AA?5?$AAi?$AAm?$AAp?$AAl?$AAe@ 100019f8     pmicsdk:mc34704sdk.obj
 0001:00000a48       ??_C@_1EO@DOFMHDHF@?$AAR?$AAe?$AAg?$AAu?$AAl?$AAa?$AAt?$AAo?$AAr?$AA?5?$AA5?$AA?5?$AAm?$AAa?$AAn?$AAa?$AAg?$AAe?$AAm?$AAe?$AAn?$AAt?$AA?5?$AAn?$AAo?$AAt?$AA?5?$AAi?$AAm?$AAp?$AAl?$AAe@ 10001a48     pmicsdk:mc34704sdk.obj
 0001:00000a98       ??_C@_1EO@HEJLHMOG@?$AAR?$AAe?$AAg?$AAu?$AAl?$AAa?$AAt?$AAo?$AAr?$AA?5?$AA4?$AA?5?$AAm?$AAa?$AAn?$AAa?$AAg?$AAe?$AAm?$AAe?$AAn?$AAt?$AA?5?$AAn?$AAo?$AAt?$AA?5?$AAi?$AAm?$AAp?$AAl?$AAe@ 10001a98     pmicsdk:mc34704sdk.obj
 0001:00000ae8       ??_C@_1EO@BBHIFLMN@?$AAR?$AAe?$AAg?$AAu?$AAl?$AAa?$AAt?$AAo?$AAr?$AA?5?$AA2?$AA?5?$AAm?$AAa?$AAn?$AAa?$AAg?$AAe?$AAm?$AAe?$AAn?$AAt?$AA?5?$AAn?$AAo?$AAt?$AA?5?$AAi?$AAm?$AAp?$AAl?$AAe@ 10001ae8     pmicsdk:mc34704sdk.obj
 0001:00000b38       ??_C@_1EO@MODBELHI@?$AAR?$AAe?$AAg?$AAu?$AAl?$AAa?$AAt?$AAo?$AAr?$AA?5?$AA1?$AA?5?$AAm?$AAa?$AAn?$AAa?$AAg?$AAe?$AAm?$AAe?$AAn?$AAt?$AA?5?$AAn?$AAo?$AAt?$AA?5?$AAi?$AAm?$AAp?$AAl?$AAe@ 10001b38     pmicsdk:mc34704sdk.obj
 0001:00000bb4       DvfcInitVoltageSupplies    10001bb4 f   voltctrl.obj
 0001:00000c98       DvfcConvertVoltage         10001c98 f   voltctrl.obj
 0001:00000dbc       DvfcUpdateSupplyVoltage    10001dbc f   voltctrl.obj
 0001:00000f50       DllEntry                   10001f50 f   dvfc_common_topaz_v1:dvfc.obj
 0001:00000f90       DVF_Init                   10001f90 f   dvfc_common_topaz_v1:dvfc.obj
 0001:000012ac       DVF_Deinit                 100022ac f   dvfc_common_topaz_v1:dvfc.obj
 0001:000012dc       DVF_Open                   100022dc f   dvfc_common_topaz_v1:dvfc.obj
 0001:00001304       DVF_Close                  10002304 f   dvfc_common_topaz_v1:dvfc.obj
 0001:00001334       DVF_IOControl              10002334 f   dvfc_common_topaz_v1:dvfc.obj
 0001:00001678       GetCurrentThread           10002678 f i dvfc_common_topaz_v1:dvfc.obj
 0001:00001690       BSPDvfcGetThreadPriority   10002690 f   dvfc:dvfc.obj
 0001:000016b0       DvfcMapDevPwrStateToSetpoint 100026b0 f   dvfc:dvfc.obj
 0001:0000174c       BSPDvfcGetSupportedDx      1000274c f   dvfc:dvfc.obj
 0001:00001764       BSPDvfcPowerGet            10002764 f   dvfc:dvfc.obj
 0001:000017d8       BSPDvfcPowerSet            100027d8 f   dvfc:dvfc.obj
 0001:000018f0       DvfcUpdateSetpoint         100028f0 f   dvfc:dvfc.obj
 0001:00001a4c       BSPDvfcIntrServ            10002a4c f   dvfc:dvfc.obj
 0001:00001a9c       BSPDvfcInit                10002a9c f   dvfc:dvfc.obj
 0001:00002144       BSPDvfcDeinit              10003144 f   dvfc:dvfc.obj
 0001:0000215c       SetEvent                   1000315c f i dvfc:dvfc.obj
 0001:00002194       NKDbgPrintfW               10003194 f   coredll:COREDLL.dll
 0001:000021a4       DisableThreadLibraryCalls  100031a4 f   coredll:COREDLL.dll
 0001:000021b4       CreateThread               100031b4 f   coredll:COREDLL.dll
 0001:000021c4       InterruptInitialize        100031c4 f   coredll:COREDLL.dll
 0001:000021d4       KernelIoControl            100031d4 f   coredll:COREDLL.dll
 0001:000021e4       CreateEventW               100031e4 f   coredll:COREDLL.dll
 0001:000021f4       RegCloseKey                100031f4 f   coredll:COREDLL.dll
 0001:00002204       RegQueryValueExW           10003204 f   coredll:COREDLL.dll
 0001:00002214       OpenDeviceKey              10003214 f   coredll:COREDLL.dll
 0001:00002224       SetLastError               10003224 f   coredll:COREDLL.dll
 0001:00002234       InterruptDone              10003234 f   coredll:COREDLL.dll
 0001:00002244       WaitForSingleObject        10003244 f   coredll:COREDLL.dll
 0001:00002254       CeSetThreadPriority        10003254 f   coredll:COREDLL.dll
 0001:00002264       QueryPerformanceFrequency  10003264 f   coredll:COREDLL.dll
 0001:00002274       QueryPerformanceCounter    10003274 f   coredll:COREDLL.dll
 0001:00002284       EventModify                10003284 f   coredll:COREDLL.dll
 0001:00002294       MmMapIoSpace               10003294 f   ceddk:CEDDK.dll
 0001:000022a4       DDKClockSetpointRequest    100032a4 f   cspddk:CSPDDK.dll
 0001:000022b4       DDKClockSetpointRelease    100032b4 f   cspddk:CSPDDK.dll
 0001:000022c4       DDKClockGetSharedConfig    100032c4 f   cspddk:CSPDDK.dll
 0001:000022d4       DDKClockUnlock             100032d4 f   cspddk:CSPDDK.dll
 0001:000022e4       DDKClockLock               100032e4 f   cspddk:CSPDDK.dll
 0001:000022f4       PmicOpen                   100032f4 f   pmicsdk:mc34704sdk.obj
 0001:0000236c       PmicClose                  1000336c f   pmicsdk:mc34704sdk.obj
 0001:00002398       PmicEnable                 10003398 f   pmicsdk:mc34704sdk.obj
 0001:000023e0       PmicRegulatorSetVoltageLevel 100033e0 f   pmicsdk:mc34704sdk.obj
 0001:00002554       PmicRegulatorGetVoltageLevel 10003554 f   pmicsdk:mc34704sdk.obj
 0001:000026e4       PmicSetRegister            100036e4 f   pmicsdk:mc34704sdk.obj
 0001:000027d4       PmicGetRegister            100037d4 f   pmicsdk:mc34704sdk.obj
 0001:000028a8       DllMain                    100038a8 f   corelib0:dllmain.obj
 0001:000028e4       _DllMainCRTStartup         100038e4 f   corelib0:pegdmain.obj
 0001:00002a8c       __security_init_cookie     10003a8c f   corelib0:seccinit.obj
 0001:00002b54       exit                       10003b54 f   corelib0:cexit.obj
 0001:00002cd4       _exit                      10003cd4 f   corelib0:cexit.obj
 0001:00002cf8       _cexit                     10003cf8 f   corelib0:cexit.obj
 0001:00002d14       _c_exit                    10003d14 f   corelib0:cexit.obj
 0001:00002d30       GetCurrentProcess          10003d30 f i corelib0:cexit.obj
 0001:00002d48       _initterm                  10003d48 f   corelib0:crt0dat.obj
 0001:00002d9c       _cinit                     10003d9c f   corelib0:crt0dat.obj
 0001:00002dd8       _onexit                    10003dd8 f   corelib0:onexit.obj
 0001:000030dc       atexit                     100040dc f   corelib0:onexit.obj
 0001:00003130       memset                     10004130 f   corelib1:COREDLL.dll
 0001:00003140       __C_specific_handler       10004140 f   corelib1:COREDLL.dll
 0001:00003150       __rt_sdiv64by64            10004150 f   corelib1:COREDLL.dll
 0001:00003160       _XcptFilter                10004160 f   corelib1:COREDLL.dll
 0001:00003170       __security_gen_cookie2     10004170 f   corelib1:COREDLL.dll
 0001:00003180       free                       10004180 f   corelib1:COREDLL.dll
 0001:00003190       malloc                     10004190 f   corelib1:COREDLL.dll
 0001:000031a0       realloc                    100041a0 f   corelib1:COREDLL.dll
 0001:000031b0       _msize                     100041b0 f   corelib1:COREDLL.dll
 0001:000031c0       CloseHandle                100041c0 f   coredll:COREDLL.dll
 0001:000031d0       DeleteCriticalSection      100041d0 f   coredll:COREDLL.dll
 0001:000031e0       InterlockedExchange        100041e0 f   coredll:COREDLL.dll
 0001:000031f0       TerminateProcess           100041f0 f   coredll:COREDLL.dll
 0001:00003200       EnterCriticalSection       10004200 f   coredll:COREDLL.dll
 0001:00003210       InterlockedCompareExchange 10004210 f   coredll:COREDLL.dll
 0001:00003220       InitializeCriticalSection  10004220 f   coredll:COREDLL.dll
 0001:00003230       LeaveCriticalSection       10004230 f   coredll:COREDLL.dll
 0001:00003240       I2COpenHandle              10004240 f   i2csdk:I2CSDK.dll
 0001:00003250       I2CTransfer                10004250 f   i2csdk:I2CSDK.dll
 0001:00003260       I2CSetFrequency            10004260 f   i2csdk:I2CSDK.dll
 0001:000032cc       __IMPORT_DESCRIPTOR_COREDLL 100042cc     coredll:COREDLL.dll
 0001:000032e0       __IMPORT_DESCRIPTOR_CEDDK  100042e0     ceddk:CEDDK.dll
 0001:000032f4       __IMPORT_DESCRIPTOR_CSPDDK 100042f4     cspddk:CSPDDK.dll
 0001:00003308       __IMPORT_DESCRIPTOR_I2CSDK 10004308     i2csdk:I2CSDK.dll
 0001:0000331c       __NULL_IMPORT_DESCRIPTOR   1000431c     coredll:COREDLL.dll
 0002:00000000       __imp_MmMapIoSpace         10005000     ceddk:CEDDK.dll
 0002:00000004       \177CEDDK_NULL_THUNK_DATA  10005004     ceddk:CEDDK.dll
 0002:00000008       __imp_CreateThread         10005008     coredll:COREDLL.dll
 0002:0000000c       __imp_InterruptInitialize  1000500c     coredll:COREDLL.dll
 0002:00000010       __imp_KernelIoControl      10005010     coredll:COREDLL.dll
 0002:00000014       __imp_CreateEventW         10005014     coredll:COREDLL.dll
 0002:00000018       __imp_RegCloseKey          10005018     coredll:COREDLL.dll
 0002:0000001c       __imp_RegQueryValueExW     1000501c     coredll:COREDLL.dll
 0002:00000020       __imp_OpenDeviceKey        10005020     coredll:COREDLL.dll
 0002:00000024       __imp_DisableThreadLibraryCalls 10005024     coredll:COREDLL.dll
 0002:00000028       __imp_InterruptDone        10005028     coredll:COREDLL.dll
 0002:0000002c       __imp_WaitForSingleObject  1000502c     coredll:COREDLL.dll
 0002:00000030       __imp_CeSetThreadPriority  10005030     coredll:COREDLL.dll
 0002:00000034       __imp_QueryPerformanceFrequency 10005034     coredll:COREDLL.dll
 0002:00000038       __imp_QueryPerformanceCounter 10005038     coredll:COREDLL.dll
 0002:0000003c       __imp_EventModify          1000503c     coredll:COREDLL.dll
 0002:00000040       __imp_SetLastError         10005040     coredll:COREDLL.dll
 0002:00000044       __imp_NKDbgPrintfW         10005044     coredll:COREDLL.dll
 0002:00000048       __imp_InitializeCriticalSection 10005048     coredll:COREDLL.dll
 0002:0000004c       __imp_InterlockedCompareExchange 1000504c     coredll:COREDLL.dll
 0002:00000050       __imp_LeaveCriticalSection 10005050     coredll:COREDLL.dll
 0002:00000054       __imp_EnterCriticalSection 10005054     coredll:COREDLL.dll
 0002:00000058       __imp_TerminateProcess     10005058     coredll:COREDLL.dll
 0002:0000005c       __imp_InterlockedExchange  1000505c     coredll:COREDLL.dll
 0002:00000060       __imp_memset               10005060     corelib1:COREDLL.dll
 0002:00000064       __imp___C_specific_handler 10005064     corelib1:COREDLL.dll
 0002:00000068       __imp___rt_sdiv64by64      10005068     corelib1:COREDLL.dll
 0002:0000006c       __imp__XcptFilter          1000506c     corelib1:COREDLL.dll
 0002:00000070       __imp___security_gen_cookie2 10005070     corelib1:COREDLL.dll
 0002:00000074       __imp_free                 10005074     corelib1:COREDLL.dll
 0002:00000078       __imp_malloc               10005078     corelib1:COREDLL.dll
 0002:0000007c       __imp_realloc              1000507c     corelib1:COREDLL.dll
 0002:00000080       __imp__msize               10005080     corelib1:COREDLL.dll
 0002:00000084       __imp_CloseHandle          10005084     coredll:COREDLL.dll
 0002:00000088       __imp_DeleteCriticalSection 10005088     coredll:COREDLL.dll
 0002:0000008c       \177COREDLL_NULL_THUNK_DATA 1000508c     coredll:COREDLL.dll
 0002:00000090       __imp_DDKClockLock         10005090     cspddk:CSPDDK.dll
 0002:00000094       __imp_DDKClockUnlock       10005094     cspddk:CSPDDK.dll
 0002:00000098       __imp_DDKClockSetpointRelease 10005098     cspddk:CSPDDK.dll
 0002:0000009c       __imp_DDKClockSetpointRequest 1000509c     cspddk:CSPDDK.dll
 0002:000000a0       __imp_DDKClockGetSharedConfig 100050a0     cspddk:CSPDDK.dll
 0002:000000a4       \177CSPDDK_NULL_THUNK_DATA 100050a4     cspddk:CSPDDK.dll
 0002:000000a8       __imp_I2CTransfer          100050a8     i2csdk:I2CSDK.dll
 0002:000000ac       __imp_I2CSetFrequency      100050ac     i2csdk:I2CSDK.dll
 0002:000000b0       __imp_I2COpenHandle        100050b0     i2csdk:I2CSDK.dll
 0002:000000b4       \177I2CSDK_NULL_THUNK_DATA 100050b4     i2csdk:I2CSDK.dll
 0002:000000b8       g_DvfcIrq                  100050b8     dvfc:dvfc.obj
 0002:00000114       __security_cookie          10005114     corelib0:seccinit.obj
 0002:00000118       __security_cookie_complement 10005118     corelib0:seccinit.obj
 0002:00000164       _exitflag                  10005164     corelib0:cexit.obj
 0002:00000168       g_pCRM                     10005168     <common>
 0002:0000016c       __onexitend                1000516c     <common>
 0002:00000170       __onexitbegin              10005170     <common>
 0002:00000174       g_pcsExit                  10005174     <common>
 0002:00000178       _pRawDllMain               10005178     <common>

 entry point at        0001:000028e4

 Static symbols

 0001:000015e0       DvfcIntrServThread         100025e0 f   dvfc_common_topaz_v1:dvfc.obj
 0001:00001d7c       DvfcWorkerThread           10002d7c f   dvfc:dvfc.obj
 0001:00002938       _DllMainCRTStartupHelper   10003938 f   corelib0:pegdmain.obj
 0001:00002b78       doexit                     10003b78 f   corelib0:cexit.obj
 0001:00002e34       lockexit                   10003e34 f   corelib0:onexit.obj
 0001:00002ed0       unlockexit                 10003ed0 f   corelib0:onexit.obj
 0001:00002efc       _onexit_nolock             10003efc f   corelib0:onexit.obj
